:020000040800F2
:100000000006012001020008950E0008990E000864
:10001000ED0E0008990E0008C10E0008030200084A
:10002000030200080302000803020008C5300008AC
:10003000030200080302000803020008030200088C
:10004000030200080302000803020008030200087C
:100050000302000803020008213300084D330008A2
:1000600079330008A5330008D133000803020008E3
:10007000030200080302000803020008030200084C
:10008000030200080302000803020008030200083C
:10009000030200080302000803020008FD33000801
:1000A000030200080302000803020008030200081C
:1000B000453100080302000803020008030200089B
:1000C00003020008030200080302000803020008FC
:1000D00003020008030200080302000803020008EC
:1000E0006534000803020008030200080302000848
:1000F00003020008030200080302000803020008CC
:1001000003020008030200080302000803020008BB
:1001100003020008030200080302000803020008AB
:10012000030200080302000803020008030200089B
:10013000030200080302000803020008030200088B
:10014000030200080302000803020008F128000867
:10015000030200080302000803020008030200086B
:10016000030200080302000803020008030200085B
:10017000030200080302000803020008030200084B
:10018000030200080302000803020008030200083B
:10019000030200080302000803020008030200082B
:1001A000030200080302000803020008030200081B
:1001B000030200080302000803020008030200080B
:1001C00003020008030200080302000803020008FB
:1001D00003020008030200080302000803020008EB
:1001E00003020008030200080302000803020008DB
:1001F00003020008030200080302000803020008CB
:1002000002E000F000F8FEE772B6394880F3088893
:10021000384880F3098838484EF60851CEF200017C
:10022000086040F20000CCF200004EF63471CEF2CD
:1002300000010860BFF34F8FBFF36F8F40F20000E3
:10024000C0F2F0004EF68851CEF200010860BFF314
:100250004F8FBFF36F8F4FF00000E1EE100A4EF6A4
:100260003C71CEF200010860062080F31488BFF3D1
:100270006F8F01F0C1FF02F0ADFE4FF055301F4906
:100280001B4A91423CBF41F8040BFAE71C49194A4A
:1002900091423CBF41F8040BFAE71A491A4A1B4B3A
:1002A0009A423EBF51F8040B42F8040BF8E70020D5
:1002B0001749184A91423CBF41F8040BFAE701F094
:1002C000DFFF02F0F1FE144C144DAC4203DA54F897
:1002D000041B8847F9E700F03FF8114C114DAC4280
:1002E00003DA54F8041B8847F9E701F0C7BF0000A0
:1002F000000601200022012000000008000001206B
:100300000006012070380008002201205022012040
:1003100050220120442E01200002000800020008A3
:1003200000020008000200082DE9F04F2DED108AB0
:10033000C1F80CD0D0F80CD0BDEC108ABDE8F08F1D
:10034000002383F311882846A047002001F0D8FB42
:1003500001F0EEFA00DFFEE71B4B7B2270B51A704E
:100360006FF07F0200245A720E225C709C70DC7069
:100370001C715C719C71DC711C729A72DC7201F0F0
:10038000FDFE064601F032FF054650B90F4B9E4276
:1003900017D001339E4241F2883412BF0546002433
:1003A0000125002001F0F4FE0DB100F05BF800F033
:1003B00045FD00F0E1FB204600F0F6F800F052F8B1
:1003C000F9E70446EDE700BF50220120010007B025
:1003D00008B500F073FBA0F120035842584108BD56
:1003E00007B5054B02211B88ADF8043001A800F0C9
:1003F000B3FB03B05DF804FB4835000810B572B6D6
:10040000202383F3118862B61248C3680BB101F050
:10041000FFFB0023104A0F484FF47A7101F0BCFB38
:10042000002383F311880D4C236813B12368013B2B
:100430002360636813B16368013B6360084B1B78FA
:1004400033B9636823B9022000F066FC322363608D
:1004500010BD00BF5C220120FD03000878230120AD
:10046000702201202DE9F041454B464953F8042FF5
:10047000013201D1BDE8F0818B42F7D1424C434BB0
:1004800022689A427AD9424B9B6803F1006303F5D4
:10049000C0339A4272D2002000F08AFB3D4B02200A
:1004A000187000F031FC3C4B1A6C00221A64196E73
:1004B0001A66196E596C5A64596E5A66596E5969A2
:1004C00041F080015961596921F0800159615969F0
:1004D000196941F000511961196921F00051196140
:1004E0001B6972B62D492E4B0B601D682468BFF343
:1004F0004F8FBFF36F8F2B4BC3F88420BFF34F8F09
:100500005A6922F480325A61BFF34F8FD3F88020AA
:10051000C2F3C906C2F34E325201B70743F6E07E7A
:1005200002EA0E0838463146013948EA000CB1F1BA
:10053000FF3FC3F874C200F14040F5D1203A12F1F8
:10054000200FEDD1BFF34F8FBFF36F8FBFF34F8FEE
:10055000BFF36F8F5A6922F400325A610022C3F848
:100560005022BFF34F8FBFF36F8F72B6202383F3F8
:10057000118862B6AD4685F308882047BDE8F08152
:10058000FC7F01081C80010804800108FF7F01082E
:1005900050220120702201200038024008ED00E0C6
:1005A0000080010800ED00E02DE9F04F99B0B44C57
:1005B00001902022FF2110A8A66800F0E1FBB14ABB
:1005C0001378A346B3B9B04801211170C36072B665
:1005D000202383F3118862B6C3680BB101F018FBC6
:1005E0000023AA4AA8484FF47A7101F0D5FA0023F3
:1005F00083F31188019B13B1A54B019A1A60A54A98
:10060000A349019F0292002313704B6099461C4638
:100610001D469846012000F077FB002F00F0128263
:100620009B4B1B68002B40F00D8219B0BDE8F08F8A
:100630000220FFF7CDFE002840F0FB81019BB9F1BD
:10064000000F08BF1F46944B1B88ADF82C300221C9
:100650000BA800F081FADDE74FF47A7000F02EFA73
:10066000031E0393EADB0220FFF7B2FE8246002856
:10067000E4D0039B581E042800F2DD81DFE800F07F
:10068000030E1114170018A8052340F8343D042167
:1006900000F062FA54464FF0000856E00421784812
:1006A000F6E704217D48F3E704217D48F0E71C24A8
:1006B000204600F07FFA04340B9004210BA800F0D0
:1006C0004BFA2C2CF4D1E5E7002DB7D0002CB5D097
:1006D0000220FFF77DFE0546002800F0AF810120D3
:1006E0006C4C00F065FA0220207000F00DFB4FF01A
:1006F00000095FFA89FA504600F06AFA074658B1D5
:10070000504600F075FA09F101090028F1D12C4694
:10071000A9460027634B97E701230220237000F0CE
:10072000E9FA3E46DBF808309E4206D2304600F039
:1007300041FA0130EBD10436F4E7029B00261E702B
:10074000534BA9465E602C46374600F06DFB15B151
:10075000002C18BF0027FFF743FE5BE7002D3FF496
:100760006DAF002C3FF46AAF029B0220187000F0BE
:10077000CBFA322000F0A2F9B0F1000AC0F25E819B
:100780001AF0030540F05A81DBF8082006EB0A0353
:10079000934200F25381BAF5807F00F24F815545B4
:1007A0000DDA4FF47A7000F089F90490049B002B65
:1007B000C0F244813C4A049BAB540135EFE7C820AA
:1007C000FFF706FE0546002800F038811F2E11D8DD
:1007D000C6F12004544528BF544610AB26F0030050
:1007E00022463149184400F0A1FA2246FF212E4842
:1007F00000F0C6FA4FEAAA0A5FFA8AF22A4930469E
:1008000000F0C6FA0446002800F01A8106EB8A06BA
:1008100005469AE70220FFF7DBFD00283FF40EAF04
:1008200000F00CFA00283FF409AF4FF0000A5346DD
:10083000DBF8082092451CD2BAF11F0F12D8109A8B
:1008400001320FD02AF0030218A90A4452F8202CD2
:100850000B92184604220BA900F05CFB0AF1040A73
:100860000346E5E75046039300F0A4F9039B0B9081
:10087000EFE718A8042140F84C3D00F06DF964E75B
:1008800050220120742301205C220120FD03000876
:1008900078230120702201204A35000854220120CB
:1008A000582201204C3500087422012018A800238A
:1008B00040F8343D642100F02BF900287FF4BEAEEF
:1008C0000220FFF785FD00283FF4B8AE0B9800F03A
:1008D000A1F918AB43F8480D04211846CDE718A834
:1008E000002340F8343D642100F012F900287FF421
:1008F000A5AE0220FFF76CFD00283FF49FAE0B98D9
:1009000000F096F918AB43F8440DE5E70220FFF735
:100910005FFD00283FF492AE00F0A0F918AB43F859
:10092000400DD9E70220FFF753FD00283FF486AEC3
:100930000BA9142000F098F9824618A8042140F869
:100940003CAD00F009F951460BA896E7322000F0C3
:10095000B5F8B0F1000AFFF671AE1AF0030F7FF49C
:100960006DAEDBF808200AEB080393423FF666AE53
:100970000220FFF72DFD00283FF460AE2AF0030AA5
:10098000C244D0453FF4E1AE404600F013F90421E3
:100990000A900AA800F0E0F808F10408F1E74FF423
:1009A0007A70FFF715FD00283FF448AE00F046F9D5
:1009B00000283FF4AFAE109B01330CD0082210A9E1
:1009C000002000F0E5F900283FF4A4AE2022FF212A
:1009D00010A800F0D5F9FFF703FD374801F098F8AB
:1009E00023E6002D3FF42AAE002C3FF427AE18A8D2
:1009F000002340F8343D642100F08AF88246002844
:100A00007FF41CAE0220FFF7E3FC00283FF416AE93
:100A10000390FFF7E5FC41F2883001F079F80B987C
:100A200000F036FA00F000FA039B57461C461D46BC
:100A3000F0E5054689E64FF00008FFE52546FDE5AF
:100A40002C4667E6002000F039F80490049B002B48
:100A5000FFF6E3AD012000F04DF9049B213B122B82
:100A60003FF6D8AD01A252F823F000BF31060008CE
:100A700059060008C90600081506000815060008F2
:100A8000150600085D0700084D0900081508000854
:100A9000AD080008DF0800080D0900081506000869
:100AA00025090008150600089F0900084B070008E3
:100AB00015060008E3090008A086010037B5114BB0
:100AC0001A780132D2B20024012A01468DF807407B
:100AD00011D80D4803681D6A4FF47A734B43012205
:100AE0000DF10701A847012805D1084B9DF8070023
:100AF0001C7003B030BD4FF4FA7001F009F84FF0EC
:100B0000FF30F6E70022012068260120AC230120F7
:100B100038B50E4B1A780132D2B2012A05460ED8EA
:100B20000B4803681C6A4FF47A734B43042229462E
:100B3000A047042803D1074B0020187038BD4FF49C
:100B4000FA7000F0E5FF4FF0FF3038BD00220120C1
:100B500068260120AC23012030B4054C2368DD69F0
:100B6000044B0A46AC460146204630BC604700BFF5
:100B700068260120A0860100F8B501F003FA094CAF
:100B8000094E0A4F2070002530682378834207D928
:100B900001F0F2F9336805440133BD423360F3D903
:100BA000F8BD00BFAD23012080230120FF7F01009D
:100BB00001F096BA00F1006000F5C030006870479F
:100BC00000F10060920000F5C03001F021BA000091
:100BD000054B1A68054B1B789B1A834202D91044B7
:100BE00001F0CAB90020704780230120AD23012005
:100BF00038B5074D04462868204401F0C5F928B9E6
:100C000028682044BDE8384001F0D6B938BD00BF9F
:100C10008023012010F0030308D1B0F5806F05D8C0
:100C200000F10050A0F57120006870470020704767
:100C3000014BC058704700BF20F4F01F064991F8DF
:100C4000243033B100230822086A81F82430FFF7EA
:100C5000B7BF0120704700BF84230120014B1868F3
:100C6000704700BF002004E0F0B5204B1E68204B09
:100C70001F885D6893F90840C6F30B02BA424FEA39
:100C8000164622D09F89BA4221D01F8BBA4206D184
:100C900002220C2404FB02335D6893F90840B6F588
:100CA000805F16D041F201039E4208BF5A24421EC3
:100CB0000A44013D0B46934215D215F9016F581CA9
:100CC0004EB1034600F8016CF5E70022E1E701228E
:100CD000DFE74124EBE72C2582421D7001D9981CE7
:100CE0005C70401AF0BD1846FBE700BF002004E02E
:100CF00004220120022802BF024B4FF480229A6195
:100D0000704700BF00000240022802BF014B0422CE
:100D10009A61704700000240022801BF024A5369ED
:100D200083F00403536170470000024010B50023B4
:100D3000934203D0CC5CC4540133F9E710BD0000EA
:100D400030B5441E14F9010F0B4660B193F9005001
:100D5000854201F1010106D11AB993F90020801AE8
:100D600030BD013AEEE7002AF7D1104630BD000051
:100D700002460346981A13F9011B0029FAD170475D
:100D800002440346934202D003F8011BFAE770477E
:100D90002DE9F047234C94F8243005468846174641
:100DA00083BB2E46DFF87C90C7B394F824302BB970
:100DB0002022FF2148462662FFF7E2FF94F8240034
:100DC000C0F10805BD4228BF3D465FFA85FAAD0077
:100DD00041462A4604EB8000FFF7A8FF94F8243030
:100DE000A7EB0A079A445FFA8AFABAF1080F2E4471
:100DF000A844FFB284F824A0D6D1FFF71FFF002833
:100E0000D2D108E0266A06EB8306B042CAD0FFF7CB
:100E100015FF0028C5D10020BDE8F0870120BDE8FE
:100E2000F08700BF84230120024B1A78024B1A700E
:100E3000704700BFAC2301200022012038B5104DBF
:100E4000104C284600F008F92146284600F030F9F9
:100E500024680D48E26ED2F8043843F00203C2F869
:100E6000043800F055FE0949204600F035FAE26EDC
:100E7000D2F8043823F00203C2F8043838BD00BFAA
:100E8000682601202036000840420F00483600083E
:100E900070470000FEE7000000B59BB0EFF309814A
:100EA00068226846FFF742FFEFF30583034B9A6B16
:100EB0009A6A9A6A9A6A9A6A9B6AFEE700ED00E06B
:100EC00000B59BB0EFF3098168226846FFF72EFF5B
:100ED000EFF30583044B9A6B9A6A9A6A9A6A9A6A44
:100EE0009A6A9B6AFEE700BF00ED00E000B59BB088
:100EF000EFF3098168226846FFF718FFEFF30583D7
:100F0000034B5A6B9A6A9A6A9A6A9A6A9B6AFEE7D4
:100F100000ED00E030B5084D0A4491420BD011F8C5
:100F2000013B09245840013CF7D040F300032B401B
:100F300083EA5000F7E730BD2083B8ED0023044971
:100F40001A465A50C8180833802B4260F9D17047AE
:100F5000B023012072B6202383F3118862B6704754
:100F6000026843681143016003B1184770470000ED
:100F700013B5446BD4F894341A681178042915D148
:100F8000217C022912D11979128901238B40134245
:100F90000CD101A904F14C0001F026FFD4F89444CF
:100FA000019B21790246206800F0E6F902B010BDED
:100FB000143001F0ABBE00004FF0FF33143001F0ED
:100FC000A5BE00004C3001F07BBF00004FF0FF33A6
:100FD0004C3001F075BF0000143001F07BBE000002
:100FE0004FF0FF31143001F075BE00004C3001F0BD
:100FF00047BF00004FF0FF324C3001F041BF00000E
:10100000D0F8942438B5136819780429054601D01E
:10101000012038BD017C0229FAD112795C890120B6
:1010200090400440F4D105F1140001F00DFE024699
:101030000028EDD0D5F894544FF48073286869796E
:1010400000F088F9204638BD406BFFF7D9BF00009B
:1010500000207047704700007FB5124B03600023EB
:1010600043608360C360012502260F4B057404466C
:101070000290019300F18402294600964FF4807398
:10108000143001F0BDFD094B0193029400964FF41A
:10109000807304F52372294604F14C0001F080FEB0
:1010A00004B070BD7C35000849100008710F0008BD
:1010B00008B50A68FFF74EFF0B7902EB830318624D
:1010C0004B790D3342F823008B7913B102EB830285
:1010D000106202230374C0F89414002383F3118870
:1010E00008BD000038B5037F044613B190F85430B2
:1010F000ABB9201D01250221FFF732FF04F11400D6
:1011000025776FF0010100F02BFD84F8545004F1B5
:101110004C006FF00101BDE8384000F021BD38BD42
:1011200010B5012104460430FFF71AFF002323778E
:1011300084F8543010BD000038B504460025143042
:1011400001F076FD04F14C00257701F041FE201DF1
:1011500084F854500121FFF703FF2046BDE83840D2
:10116000FFF74EBF90F85C3003F06003202B19D1DD
:1011700090F85D20212A0AD0222A4FF000030ED0D9
:10118000202A0FD1084A02650722426504E0064B77
:1011900003650723436500238365012070470365CA
:1011A0004365F9E70020704728220120D0F89434E5
:1011B00037B51A681178042904461AD1017C02292E
:1011C00017D11979128901238B40134211D100F1F3
:1011D0004C05284601F0BAFE58B101A9284601F095
:1011E00003FED4F89444019B21790246206800F064
:1011F000C3F803B030BD000000EB8103F7B51C6AF3
:1012000005460E46ECB105EB8607FFF7A3FE201D51
:101210000821FFF7A5FEFB685B691B684C3413B11E
:10122000204601F0EFFD01A9204601F0DDFD024658
:1012300048B1019B3146284600F09EF8002383F315
:10124000118803B0F0BDFB685A691268002AF5D016
:101250001B8A013B1340F1D105F15C02EAE7000073
:101260000D3138B550F82140D4B1FFF773FED4F8F2
:1012700094241368527903EB8203DB689B695D68F1
:1012800045B104216018FFF76BFE294604F11400F4
:1012900001F0E4FC2046FFF7B3FE002383F311883E
:1012A00038BD00007047000072B6202383F3118818
:1012B00062B6704701F06AB80123037000234360EF
:1012C00000F1240200F1380142F8043B8A42136124
:1012D000FAD103814381704738B50446FFF7E4FF34
:1012E00000254160C560056145618561C561056294
:1012F00001F05CF80223237085F3118838BD0000EB
:1013000070B500EB810305465069DA600E4614465D
:1013100018B110220021FFF733FDA06918B1102287
:101320000021FFF72DFD31462846BDE8704001F051
:1013300007B90000028902F001020281428902F02D
:10134000010242810022026142618261C261026245
:1013500001F08AB9F0B400EB81044789E468012503
:10136000A4698D403D43458123600023A2606360F2
:10137000F0BC01F0A5B90000F0B400EB81040789CE
:10138000E468012564698D403D43058123600023A5
:10139000A2606360F0BC01F021BA000070B50223C6
:1013A000002504460370A0F8645080F8665080F869
:1013B000675005814581C560056145618561C561ED
:1013C000056280F84C5001F057F863681B6823B140
:1013D00029462046BDE87040184770BD4368027832
:1013E0001B6880F86820052202700BB104211847A1
:1013F00070470000436890F868201B6802700BB1CA
:10140000052118477047000090F84C3070B504462D
:1014100013B1002380F84C3004F15C02204601F047
:1014200045F963689B6863BB94F85C5015F06006EF
:1014300015D194F85D3005F07F0545EA032540F2AB
:1014400002339D4200F00B8159D8022D00F0D98063
:101450003DD8002D00F08580012D00F0CC800021CA
:10146000204601F093FB0021204601F085FB6368D4
:101470001B6813B1062120469847062384F84C3098
:1014800070BD204698470028CED094F8632094F889
:10149000623043EA0223626D934238BF636594F978
:1014A0005C30656D002B80F2FC80002D00F0EB803D
:1014B000092384F84C30FFF7F7FE636D226D00219D
:1014C0002046FFF759FF002383F3118870BDB5F55F
:1014D000817F00F0B080B5F5407F49D0B5F5807FC1
:1014E000BDD194F85E30012BB9D1B4F8643023F04B
:1014F0000203A4F8643026656665A665C5E740F278
:1015000001639D421ED8B5F5C06F3BD2B5F5A06F03
:10151000A5D1B4F85C30B3F5A06F0ED194F85E306D
:1015200084F86630204600F0FFFF63681B6813B143
:101530000121204698470323237000232365636518
:10154000A365A2E7B5F5106F32D040F602439D4285
:1015500051D0B5F5006F82D104F1670323650123F3
:1015600024E004F16403236502236365A5658CE729
:1015700094F85E30012B7FF472AFB4F8643043F01E
:101580000203B6E794F86120616894F860304D6812
:1015900094F85F1043EA0223204694F85E20A8479F
:1015A00000283FF45CAF4368236503686365A4E7E4
:1015B0002378042B0FD1FFF777FE2046FFF7BAFE02
:1015C00086F31188636884F867601B6803212170C3
:1015D0000BB12046984794F85E30002BADD084F8CC
:1015E00067300423237063681B68002BA5D0022199
:1015F00020469847A1E7374B236502236365002304
:101600009EE794F8601011F0800F204601F00F0162
:101610000ED001F03DF8012806D002287FF41FAF5C
:101620002D4B2365606568E72C4B2365656564E792
:1016300001F020F8EFE794F85E30002B7FF40FAF55
:1016400094F8603013F00F013FF477AF1A0620468C
:1016500002D501F0AFFA70E701F0A2FA6DE794F855
:101660005E30002B7FF4FBAE94F8603013F00F0176
:101670003FF463AF1B06204602D501F087FA5CE712
:1016800001F07AFA59E7142384F84C30FFF70CFE86
:101690002B462A4629462046FFF75CFE85F3118833
:1016A00070BD5DB1152384F84C30FFF7FDFD636D0F
:1016B000226D00212046FFF74DFE04E70B2384F83E
:1016C0004C30FFF7F1FD2B462A4629462046FFF70E
:1016D00053FEE3E7AC350008A4350008A835000840
:1016E00038B590F84C300446152B28D8DFE803F0C5
:1016F0003C27272727273C27270B2837272727275B
:10170000272727273C3C90F8631090F86220436D10
:1017100042EA01229A4213D9C268128AB3FBF2F557
:1017200002FB153565B9FFF7BFFD2B462A46294652
:10173000FFF722FE85F311880A2384F84C3038BD68
:10174000142384F84C30FFF7AFFD00231A461946E6
:101750002046FFF7FFFD002383F3118838BD836D1A
:1017600003B198470023E8E7002101F00FFA0021B8
:10177000204601F001FA63681B6813B10621204678
:1017800098470623D9E7000090F84C20152A38B571
:10179000044621D80123934040F6416213421CD1F4
:1017A00013F480150ED19B0216D50B2380F84C3014
:1017B000FFF77AFD2B462A462946FFF7DDFD85F324
:1017C000118838BDC3689B695B682BB9836D03B111
:1017D0009847002384F84C3038BD002101F0D6F939
:1017E0000021204601F0C8F963681B6813B1062187
:1017F000204698470623EDE7024B00221B605B6002
:101800009A60704730240120002303748268054BDE
:101810001B6899689142FBD25A680360426010606D
:10182000586070473024012008B572B6202383F336
:10183000118862B6037C032B05D0042B0DD02BB985
:1018400083F3118808BD436900221A604FF0FF330B
:101850004361FFF7D9FF0023F2E790E80C001A601C
:1018600002685360F2E70000002303748268054BAE
:101870001B6899689142FBD85A6803604260106007
:101880005860704730240120054B196908741868A6
:1018900002681A605360186101230374FEF744BDA7
:1018A0003024012030B54B1C87B005460A4C10D0BF
:1018B00023690A4A01A800F06FF92846FFF7E4FF00
:1018C000049B13B101A800F0A3F92369586907B07C
:1018D00030BDFFF7D9FFF8E73024012029180008B0
:1018E00038B50C4D41612B6981689A689142044674
:1018F00003D8BDE83840FFF787BF1846FFF784FFDD
:1019000001232C61014623742046BDE83840FEF7D0
:101910000BBD00BF30240120044B1A681B6990687E
:101920009B68984294BF002001207047302401201A
:1019300010B5084C236820691A682260546001229F
:1019400023611A74FFF790FF01462069BDE810403B
:10195000FEF7EABC30240120FEE7000010B5194C68
:10196000FFF74AFF00F00AF980221749204600F0ED
:101970008FF8012344F8180C0374144B144AD968E7
:1019800021F4E0610904090C0A431249DA60CA68CB
:1019900042F08072CA60104A1049C2F8B01F116844
:1019A00041F0010111601022DA77202283F8222011
:1019B000002383F3118862B60948BDE8104000F0A7
:1019C00089B800BF58240120B035000800ED00E0C0
:1019D0000003FA05F0ED00E0001000E055CEACC5C4
:1019E000B83500082DE9F84F204C4FF00008656924
:1019F00004F11407C1464FF08043266A5B6AAA6867
:101A00009E1B96421FD34FF0200AAA68236AD5F87E
:101A10000CB0134423622B68BB425F60A6EB020646
:101A20006361C5F80C8001D101F0BAFA89F311881D
:101A30002869D84772B68AF3118862B66569AB68BF
:101A40009E42E2D2D7E76269BA420CD09168236223
:101A50008E1B9660A86802282CBF1818981CBDE839
:101A6000F84F01F0A3BABDE8F88F00BF3024012081
:101A7000034B59685A68521A9042FBD8704700BF0E
:101A8000001000E072B6202383F3118862B670471D
:101A90008260022202740022427470478368A3F1BC
:101AA0007C0243F80C2C026943F83C2C426943F851
:101AB000382C074A43F81C2CC26843F8102C022229
:101AC00003F8082C002203F8072CA3F11800704734
:101AD0004103000810B5FFF7D5FFFFF7DFFF002136
:101AE0000446FFF7FDFE002383F31188204610BD56
:101AF000024B1B6958610F20FFF7C6BE302401203E
:101B000008B5FFF7BFFFBDE80840FFF7F1BF0000D1
:101B100008B50146FFF7B6FF0820FFF7C3FE002314
:101B200083F3118808BD000049B1064B42681B6968
:101B300018605A60136043600420FFF7B3BE4FF093
:101B4000FF307047302401200368984206D01A689D
:101B50000260506059611846FFF756BE704700009A
:101B600038B504460D462068844200D138BD03686C
:101B700023605C604561FFF747FEF4E7054B03F126
:101B800014025A619A614FF0FF32DA6100221A6240
:101B9000704700BF30240120F8B503614FF0804347
:101BA000C2605C6A194B1A46022952F8145F38BFAA
:101BB0000221954206461F460AD1586198611C626F
:101BC0000560456081600819BDE8F84001F0E0B9A2
:101BD000186AAB68241A0C1902D3E41A2D6804E0C1
:101BE0009C4202D2204401F0E1F9AB689C42F4D857
:101BF0006B68736035601E606E60B460A9684FF0FA
:101C0000FF33091BA960FB61F8BD00BF3024012030
:101C100010B41B4C234653F8141F814210D0416866
:101C200002680A60026851609A424FF00001C16088
:101C300003D0936881680B4493605DF8044B704750
:101C40000A68626100209A425360C86003D15DF85F
:101C5000044B01F0A5B993688868034493604FF082
:101C60008042206A526A121A9342E6D9991A0129CF
:101C700098BF931C18445DF8044B01F097B900BF5E
:101C80003024012000207047FEE70000704700006C
:101C90004FF0FF307047000072B6202383F31188A5
:101CA00062B67047022906D0032906D001290648EA
:101CB00018BF0020704705487047032A9ABF0448A0
:101CC00000EBC20000207047A43600085836000818
:101CD0003022012070B59AB001AD0646084629466B
:101CE000144600F091F82846FFF742F8C0B2431CB2
:101CF0005B0086E81800237003236370002302341E
:101D00001946DAB2904204F1020401D81AB070BD4B
:101D1000EA5C04F8022C04F8011C0133F1E700002E
:101D200008B5FFF7B9FF0348FFF740FA002383F334
:101D3000118808BD6826012010B50446052915D86C
:101D4000DFE801F015140315151BFFF7A5FF0E4A78
:101D50000121FFF7D5FA20460C4A0221FFF7D0FAFD
:101D60000B48FFF7E9F9002383F3118810BDFFF753
:101D700093FF0748FFF7B6F9F5E7FFF78DFF044833
:101D8000FFF7CEF9EFE700BFD8350008FC350008B3
:101D90006826012038B50C4D0C4C0D492A4604F13B
:101DA0000800FFF797FF05F1CA0204F11000094986
:101DB000FFF790FF05F5CA7204F118000649BDE867
:101DC0003840FFF787BF00BF302B012030220120B1
:101DD00028360008323600083D36000870B5044643
:101DE00008460D46FEF7C4FFC6B22046013403780C
:101DF0000BB9184670BD32462946FEF7A1FF0028F0
:101E0000F3D1012070BD00002DE9F84F05460C46C6
:101E1000FEF7AEFF2A49C6B22846FFF7DFFF08B13A
:101E20000136F6B227492846FFF7D8FF08B1103629
:101E3000F6B2632E0DD8DFF88890DFF888A0224F25
:101E4000DFF88CB0DFF88C802E7846B92670BDE8BC
:101E5000F88F29462046BDE8F84F01F06DBB252ECE
:101E600029D1072249462846FEF76AFF40B9D8F82B
:101E700000302360D8F80430636007350834E3E7A6
:101E8000082251462846FEF75BFFA0B90F4BA21C63
:101E900013F8011F09095B45C95D02F8021C197896
:101EA00001F00F0102F10202C95D02F8031CEFD13B
:101EB00018340835C8E7267001350134C4E700BF7F
:101EC000C43600083D360008D53600081FF4F01F60
:101ED0002BF4F01FCC360008BFF34F8F024AD368B3
:101EE000DB03FCD4704700BF003C024008B5074B41
:101EF0001B7853B9FFF7F0FF054B1A69002ABFBFE3
:101F0000044A5A6002F188325A6008BD8E2D0120C1
:101F1000003C02402301674508B5054B1B7833B9E7
:101F2000FFF7DAFF034A136943F00043136108BD6A
:101F30008E2D0120003C0240072870B513D80B4AB3
:101F40000B4C137863B90B4E4FF0006144F823102B
:101F500056F823500133082B2944F7D1012313707D
:101F600054F8200070BD002070BD00BFB02D0120CE
:101F7000902D0120E8360008014B53F820007047EF
:101F8000E836000808207047072810B5044601D934
:101F9000002010BDFFF7D0FF064B53F82430184443
:101FA000C21A0BB9012010BD12680132F0D1043BF6
:101FB000F6E700BFE8360008072810B5044621D828
:101FC000FFF78AFFFFF792FF0F4AF323D360C300A6
:101FD000DBB243F4007343F002031361136943F46B
:101FE00080331361FFF778FFFFF7A6FF074B53F825
:101FF000241000F0DDF8FFF78FFF2046BDE8104009
:10200000FFF7C2BF002010BD003C0240E8360008C8
:102010002DE9F84312F00103154640D18218B2F1C0
:10202000016F3CD22C4B1B6813F0010337D02B4CB3
:10203000FFF75CFFF323E360FFF74EFF40F2012759
:10204000032D01D9830713D0244C0F46401A40F2C8
:102050000118EB1B0B44012B00EB0706236924D866
:1020600023F001032361FFF757FF0120BDE8F88348
:10207000236923F44073236123693B43236151F8AF
:10208000046B0660BFF34F8FFFF726FF03689E4285
:1020900008D0236923F001032361FFF73DFF0020EF
:1020A000BDE8F883043D0430CAE723F4407323619C
:1020B000236943EA08032361B94637F8023B3380BA
:1020C000BFF34F8FFFF708FF3688B9F80030B6B27C
:1020D000B342BED0DDE700BF00380240003C024002
:1020E000084908B50B7828B153B9FFF7FFFE012363
:1020F0000B7008BD23B1BDE808400870FFF70CBFA6
:1021000008BD00BF8E2D012010B50244064B0439D6
:10211000D2B2904200D110BD441C00B253F820004E
:1021200041F8040FE0B2F4E750280040104B30B5FE
:102130001C6F240407D41C6F44F400741C671C6FCC
:1021400044F400441C670B4C236843F48073236001
:102150000244094B0439D2B2904200D130BD441C34
:1021600000B251F8045F43F82050E0B2F4E700BF3A
:1021700000380240007000405028004007B501229E
:1021800001A90020FFF7C0FF019803B05DF804FB30
:1021900013B50446FFF7F2FFA04206D002A90122C0
:1021A00041F8044D0020FFF7C1FF02B010BD000050
:1021B0000144BFF34F8F064B884204D3BFF34F8FC8
:1021C000BFF36F8F7047C3F85C022030F4E700BFA5
:1021D00000ED00E0034B1B689B0042BF024B012255
:1021E0001A70704774380240B12D0120014B1878E5
:1021F000704700BFB12D0120F0B5BFF34F8FBFF383
:102200006F8F1D4B0021C3F85012BFF34F8FBFF3E8
:102210006F8F5A6942F400325A61BFF34F8FBFF398
:102220006F8FC3F88410BFF34F8FD3F88020C2F3B1
:10223000C904C2F34E325201A50743F6E07602EA22
:10224000060E284621464EEA00070139C3F860729F
:102250004F1C00F14040F6D1203A12F1200FEED190
:10226000BFF34F8F5A6942F480325A61BFF34F8FE8
:10227000BFF36F8FF0BD00BF00ED00E0FEE7000090
:10228000084A094B09498B4204D3094A0021934269
:1022900005D3704752F8040F43F8040BF3E743F8F3
:1022A000041BF4E7BC380008442E0120442E012012
:1022B000442E0120036F30B500229D68C46E114684
:1022C0004FF0FF3004EB421301329542C3F800197E
:1022D000C3F81019C3F80809C3F8001BC3F8101B92
:1022E000C3F8080BEED24FF00113C4F81C3830BD10
:1022F000890141F02001016103699B06FCD4122091
:10230000FFF7B6BB204B03EB80022DE9F047D2F874
:102310000CE0DD6EDEF81420461CD2F800C005EBA0
:10232000063605EB4018516861450BD3D5F83428C3
:10233000012303FA00F022EA0000C5F83408184629
:10234000BDE8F087BEF81040ACEB0103A34228BF04
:102350002346D8F81849A4B2B3EB840F10D8946878
:102360001F46A4F1040959F804AFC6F800A0042FD1
:1023700001D9043FF7E71C440B4494605360D2E753
:102380000020BDE8F08700BFB42D012010B5054C3A
:102390002046FEF791FF4FF0A043E366024B236710
:1023A00010BD00BFB42D01202C3700080378012B8D
:1023B00070B5054650D12A4BC46E98421BD1294BAB
:1023C0005A6B42F080025A635A6D42F080025A659D
:1023D0005A6D5A6942F080025A615A6922F08002AD
:1023E0005A610E2143205B6900F0EEFB1E4BE36057
:1023F0001E4BC4F800380023C4F8003EC0232360FD
:10240000EE6E4FF40413A3633369002BFCDA01234F
:1024100033610C20FFF72CFB3369DB07FCD412205F
:10242000FFF726FB3369002BFCDA0026A66028465E
:10243000FFF740FF6B68C4F81068DB68C4F81468E5
:10244000C4F81C684BB90A4BA3614FF0FF336361BA
:10245000A36843F00103A36070BD064BF4E700BF1F
:10246000B42D012000380240401400400300200237
:10247000003C30C0083C30C0F8B5C46E05460021B1
:102480002046FFF735FF296F00234FF001128F68B8
:10249000C4F834384FF00066C4F81C284FF0FF3001
:1024A00004EB431201339F42C2F80069C2F8006B8B
:1024B000C2F80809C2F8080BF2D20B68EA6E6B6723
:1024C000636210231361166916F01006FBD1122007
:1024D000FFF7CEFAD4F8003823F4FE63C4F80038CE
:1024E000A36943F4402343F01003A3610923C4F814
:1024F0001038C4F814380A4BEB604FF0C043C4F8EE
:10250000103B084BC4F8003BC4F81069C4F800390C
:102510006B6F03F1100243F480136A67A362F8BD86
:102520000837000840800010C26E90F86610D2F89C
:10253000003823F4FE6343EA0113C2F80038704701
:102540002DE9F0410EB200EB86080D46D8F80C10CC
:102550000F6807F00303022B50D0032B50D03D4AE5
:102560003D4F012B18BF1746C46E4FEA451E04EBC2
:102570000E030022C3F8102B8A6905F1100C002A03
:1025800040D04A8A05F158035B013A43E2500123E7
:10259000D4F81C2803FA0CF31343A6444A69C4F880
:1025A0001C380023CEF8103905F13F03002A39D03A
:1025B0000A8A898B9208012988BF4A43416F04EB3C
:1025C0008303561841EA0242466729465A6020466C
:1025D000FFF78EFED8F80C301B8A43EA85531F4361
:1025E00005F148035B01E7500123D4F81C2803FAE6
:1025F00005F51543C4F81C58BDE8F081174FB3E743
:10260000174FB1E704EB4613D3F8002B22F4004236
:10261000C3F8002BD4F81C28012303FA0CF322EA98
:102620000303BAE704EB83030E4A5A6004EB461631
:1026300029462046FFF75CFED6F8003923F4004314
:10264000C6F80039D4F81C38012202FA05F523EA4D
:102650000505CFE7008000100080041000800810FE
:1026600000800C1000040002026F12684267FFF73E
:1026700021BE00005831C36E49015B5813F400407D
:1026800004D013F4001F14BF012002207047000083
:102690004831C36E49015B5813F4004004D013F471
:1026A000001F14BF012002207047000000EB8101D1
:1026B000CB68196A0B6813604B6853607047000061
:1026C00000EB810330B5DD68AA691368D36019B9DE
:1026D000402B84BF402313606B8A1468C26E1C4475
:1026E000013CB4FBF3F46343033323F0030302EB35
:1026F000411043EAC44343F0C043C0F8103B2B6889
:1027000003F00303012B09B20ED1D2F8083802EB13
:10271000411013F4807FD0F8003B14BF43F0805386
:1027200043F00053C0F8003B02EB4112D2F8003BEB
:1027300043F00443C2F8003B30BD00002DE9F041F6
:10274000254DEE6E06EB40130446D3F8087BC3F824
:10275000087B38070AD5D6F81438190706D505EBD3
:1027600084032146DB6828465B689847FA0731D521
:10277000D6F81438DB072DD505EB8403D968DCB90E
:102780008B69488A5E68B6FBF0F200FB12629AB968
:102790001868DA6890420FD2121A83E8140072B6F1
:1027A000202383F3118862B60B482146FFF788FF88
:1027B00084F31188BDE8F081012303FA04F26B89E8
:1027C00023EA02036B81CB6823B121460248BDE8AE
:1027D000F0411847BDE8F081B42D012000EB8103E2
:1027E00070B5DD68C36E6C692668E6604A0156BB49
:1027F0001A444FF40020C2F810092A6802F00302BC
:10280000012A0AB20ED1D3F8080803EB421410F4DF
:10281000807FD4F8000914BF40F0805040F0005091
:10282000C4F8000903EB4212D2F8000940F004405A
:10283000C2F80009D3F83408012202FA01F1014379
:10284000C3F8341870BD19B9402E84BF40202060F1
:1028500020682E8A841940F00050013C1A44B4FBD1
:10286000F6F440EAC440C6E7F8B504461F48C56E12
:1028700005EB4413D3F80869C3F80869F10719D5C3
:10288000D5F81038DA0715D500EB8403D9684B6901
:102890001F68DA6897421AD2D21B00271A605F605D
:1028A00072B6202383F3118862B62146FFF796FFA4
:1028B00087F31188330617D5D5F834280123A340B0
:1028C000134211D02046BDE8F840FFF71BBD01239D
:1028D00003FA04F2038923EA020303818B68002BC5
:1028E000E8D021469847E5E7F8BD00BFB42D0120A8
:1028F000A0482DE9F84FC56E6E69AB691E4016F40D
:10290000805F6E61044605D0FEF748FDBDE8F84FD4
:1029100000F0E8BB002E12DAD5F8003E95489B0780
:102920001EBFD5F8003E23F00303C5F8003ED5F8DE
:10293000043823F00103C5F80438FEF75BFD3705C2
:1029400002D58C48FEF74AFDB0040CD5D5F80838FE
:1029500013F0060FEB6823F470530CBF43F41053CD
:1029600043F4A053EB60310704D56368DB680BB117
:1029700080489847F2026FD4B3020CD5D4F86C802B
:10298000DFF8F0A100274FF00109236F9B68F9B22F
:102990008B4280F09C80F70619D5E16E0A6AC2F37B
:1029A0000A1702F00F0302F4F012B2F5802F00F0C4
:1029B000B680B2F5402F0AD104EB830301F58051B4
:1029C000DB68186A00231A469F4240F09C8033035C
:1029D000D5F818481DD5E70302D50020FFF7AEFE55
:1029E000A50302D50120FFF7A9FE600302D502204E
:1029F000FFF7A4FE210302D50320FFF79FFEE202AA
:102A000002D50420FFF79AFEA30202D50520FFF7A6
:102A100095FE77037FF57AAFE60702D50020FFF732
:102A200023FFA50702D50120FFF71EFF600702D58F
:102A30000220FFF719FF210702D50320FFF714FF3B
:102A4000E20602D50420FFF70FFFA3067FF55EAF75
:102A50000520FFF709FF59E7D4F86C80DFF814A1CF
:102A600000274FF00109236F9B685FFA87FB5B45E6
:102A700082D308EB4B13D3F8002902F44022B2F5BD
:102A8000802F22D1D3F80029002A1EDAD3F800299A
:102A900042F09042C3F80029D3F80029002AFBDB5A
:102AA0005946E06EFFF724FC228909FA0BF322EA6B
:102AB0000303238104EB8B03DB689B6813B1594646
:102AC000504698475846FFF71DFC0137CBE708EB07
:102AD0004112D2F8003B03F44023B3F5802F10D10C
:102AE000D2F8003B002B0CDA628909FA01F322EAE2
:102AF0000303638104EB8103DB68DB680BB15046A1
:102B00009847013741E79C0708BF0A68072B98BF21
:102B1000027003F101039CBF120A013054E7023333
:102B200004EB830201F58051526890690268D0F885
:102B300008C04068A2EB000E0022104697420AD15E
:102B400004EB830463689B699A683A449A605A6804
:102B500017445F603BE712F0030F08BF0868964513
:102B600088BF8CF8000002F1010284BF000A0CF15A
:102B7000010CE3E7B42D0120C36E03EB4111D1F842
:102B8000003B43F40013C1F8003B7047C36E03EBF6
:102B90004111D1F8003943F40013C1F800397047EE
:102BA000C36E03EB4111D1F8003B23F40013C1F8CD
:102BB000003B7047C36E03EB4111D1F8003923F499
:102BC0000013C1F80039704700F1604300F01F02A4
:102BD000400903F5614309018000C9B200F160407A
:102BE00083F8001300F5614001239340C0F8803161
:102BF0000360704772B6202383F3118862B6704772
:102C000030B5039C0172043304FB0325C361049BAC
:102C100003630021059B00604060C1604261026166
:102C20008561046242628162C162436330BD00001B
:102C30000022416A41610161C2608262C2626FF03A
:102C40000101FEF78DBF000003694269934203D181
:102C5000C2680AB100207047181D704703691960E7
:102C6000C2680132C260C26913448269036193423F
:102C700024BF436A03610021FEF766BF38B50446EE
:102C80000D46E3683BB16269131D1268A3621344E9
:102C9000E362002038BD237A33B929462046FEF787
:102CA00043FF0028EDDA38BD6FF00100FBE70000BC
:102CB000C368C269013BC3604369134482694361CD
:102CC000934224BF436A436100238362036B03B1D1
:102CD0001847704770B50446FFF78CFF866A3EB907
:102CE000FFF7CCFF054618B186F31188284670BD62
:102CF000A36AE26A13F8015BA362934202D32046FF
:102D0000FFF7D6FF002383F31188EFE72DE9F047A3
:102D100004460E4617469846FFF76CFF0025A94665
:102D2000D4F828A0BAF1000F09D141462046FFF798
:102D3000A5FF20B18AF311882846BDE8F087A16A73
:102D4000E36AA7EB050A5B1A9A4528BF9A46BAF1CF
:102D5000400F1BD9334601F1400251F8040B43F8F0
:102D6000040B9142F9D1A36A40334036A362403547
:102D7000A26AE36A9A4202D32046FFF799FF89F3D9
:102D80001188BD42D8D2FFF735FFC9E73046524619
:102D9000FDF7CCFFA36A53445644A3625544E7E7CA
:102DA00010B5029C0172043303FB0421C3610023AC
:102DB0008362C362039B0363049B00604060C46042
:102DC00042610261816104624262436310BD00009E
:102DD000026AC260426A4261026100228262C26289
:102DE0006FF00101FEF7BCBE436902699A4203D14C
:102DF000C2680AB100207047184650F8043B0B60C7
:102E000070470000C368C2690133C360436913445B
:102E100082694361934224BF436A43610021FEF704
:102E200093BE000038B504460D46E3683BB1236904
:102E30001A1DA262E2691344E362002038BD237ABE
:102E400033B929462046FEF76FFE0028EDDA38BD7B
:102E50006FF00100FBE7000003691960C268013AE6
:102E6000C260C269134482690361934224BF436A0A
:102E7000036100238362036B03B1184770470000AE
:102E800070B504460E46FFF7B5FE856A35B91146A2
:102E9000FFF7C8FF10B185F3118870BDA36A1E70DB
:102EA000A36AE26A01339342A36204D3E169204634
:102EB0000439FFF7D1FF002080F3118870BD0000B6
:102EC0002DE9F04704460D4690469946FFF792FEDD
:102ED0000026B246A76A4FB949462046FFF7A2FF2F
:102EE00020B187F311883046BDE8F087A06AE76A11
:102EF000A8EB06033F1A9F4228BF1F46402F1BD94D
:102F000005F1400355F8042B40F8042B9D42F9D1FC
:102F1000A36A4033A3624036A26AE36A9A4204D3AA
:102F2000E16920460439FFF797FF8AF31188464587
:102F3000D9D2FFF75FFECDE729463A46FDF7F6FE08
:102F4000A36A3B443D44A3623E44E5E7026943690A
:102F50009A4203D1C3681BB9184670470023FBE7A8
:102F6000836A002BF8D0043B9B1AF5D01360C3682A
:102F7000013BC360C3691A44836902619A4224BF5A
:102F8000436A0361002383620123E5E700F0F0B8A0
:102F90004FF08043002258631A610222DA607047C2
:102FA0004FF080430022DA60704700004FF080430A
:102FB000586370474B6843608B688360CB68C3601D
:102FC0000B6943614B6903628B6943620B68036061
:102FD0007047000008B5274B27481A6940F2FF7177
:102FE0000A431A611A6922F4FF6222F007021A6189
:102FF0001A691A6B0A431A631A6D0A431A651F4A43
:103000001B6D1146FFF7D6FF1D4802F11C01FFF7AB
:10301000D1FF1C4802F13801FFF7CCFF1A4802F13A
:103020005401FFF7C7FF194802F17001FFF7C2FF13
:10303000174802F18C01FFF7BDFF164802F1A80105
:10304000FFF7B8FF144802F1C401FFF7B3FF1348BC
:1030500002F1E001FFF7AEFF114802F1FC01FFF7BA
:10306000A9FF104802F58C71FFF7A4FFBDE80840E6
:1030700000F0E0B800380240000002403837000895
:103080000004024000080240000C02400010024010
:103090000014024000180240001C024000200240C0
:1030A000002402400028024008B500F035FAFEF77F
:1030B00055FCFFF78FF8BDE80840FEF76BBE000037
:1030C00070470000064A536823F001035360EFF392
:1030D0000983683383F30988002383F311887047D9
:1030E00030EF00E010B572B6202383F3118862B68A
:1030F000104B5B6813F4006318D0F1EE103AEFF355
:1031000009844FF0807344F84C3C0B4BDB6844F867
:10311000083CA4F1680383F30988FEF7FDFB18B1AE
:10312000064B44F8503C10BD054BFAE783F3118879
:1031300010BD00BF00ED00E030EF00E051030008DB
:10314000540300084FF0804310B51A6992070AD55E
:1031500000241C6172B6202383F3118862B6FEF747
:1031600041FC84F31188BDE81040FFF7BBBF0000AD
:10317000104B1A6C42F001021A641A6E42F00102FE
:103180001A660D4A1B6E936843F0010393604FF07B
:1031900080436B229A624FF0FF32DA6200229A611A
:1031A0005A63DA605A6001225A6108211A601C20B1
:1031B000FFF70ABD00380240002004E01B4B1A69EB
:1031C0006FEA42526FEA52521A611A69C2F30A0256
:1031D0001A614FF0FF301A695A69586100215A6923
:1031E00059615A691A6A62F080521A621A6A02F0C8
:1031F00080521A621A6A5A6A58625A6A59625A6A3C
:103200000B4A106840F480701060186F00F4407032
:10321000B0F5007F1EBF4FF4803018671967536800
:1032200023F40073536000F057B900BF0038024028
:1032300000700040354B4FF080521A64344A4FF40E
:10324000404111601A6842F001021A601A68920740
:10325000FCD59A6822F003029A602C4B19469A68B2
:1032600012F00C02FBD1186800F0F90018609A60A7
:103270001A6842F480321A600B689B03FCD54B6FCE
:1032800043F001034B67214B5A6F9007FCD5214A4D
:103290005A601A6842F080721A601D4B1A465968CB
:1032A0004904FCD5196841F4803119605368D8038A
:1032B000FCD5136843F400331360154A536899032F
:1032C000FCD5124B1A689201FCD5134A9A6040F261
:1032D0000112C3F88C200022C3F890200F4A40F25C
:1032E000073111609A6842F002029A60074B9A68AF
:1032F00002F00C02082AFAD15A6C42F480425A6455
:103300005A6E42F480425A665B6E70470038024043
:1033100000700040086C400900948838003C02406E
:10332000084A08B5536911680B4003F00103536163
:1033300023B1054A13680BB150689847BDE80840AF
:10334000FFF7D0BE003C0140B0230120084A08B579
:10335000536911680B4003F00203536123B1054A1E
:1033600093680BB1D0689847BDE80840FFF7BABE34
:10337000003C0140B0230120084A08B55369116898
:103380000B4003F00403536123B1054A13690BB1E9
:1033900050699847BDE80840FFF7A4BE003C0140D3
:1033A000B0230120084A08B5536911680B4003F0A7
:1033B0000803536123B1054A93690BB1D06998475B
:1033C000BDE80840FFF78EBE003C0140B02301205D
:1033D000084A08B5536911680B4003F010035361A4
:1033E00023B1054A136A0BB1506A9847BDE80840FB
:1033F000FFF778BE003C0140B0230120174B10B509
:103400005C691A68144004F478725A61A30604D502
:10341000134A936A0BB1D06A9847600604D5104AE4
:10342000136B0BB1506B9847210604D50C4A936B74
:103430000BB1D06B9847E20504D5094A136C0BB168
:10344000506C9847A30504D5054A936C0BB1D06C1A
:103450009847BDE81040FFF745BE00BF003C014063
:10346000B02301201A4B10B55C691A68144004F4AB
:103470007C425A61620504D5164A136D0BB1506D3A
:103480009847230504D5134A936D0BB1D06D984727
:10349000E00404D50F4A136E0BB1506E9847A10497
:1034A00004D50C4A936E0BB1D06E9847620404D5D4
:1034B000084A136F0BB1506F9847230404D5054A8F
:1034C000936F0BB1D06F9847BDE81040FFF70ABE6D
:1034D000003C0140B0230120062108B50846FFF753
:1034E00073FB06210720FFF76FFB06210820FFF77B
:1034F0006BFB06210920FFF767FB06210A20FFF777
:1035000063FB06211720FFF75FFB06212820BDE89B
:103510000840FFF759BB000008B5FFF74FFEFDF765
:103520000DFDFDF7C7FEFDF795FDFFF7C9FDBDE8F1
:103530000840FFF72BBD0000034611F8012B03F8EC
:10354000012B002AF9D1704712101213121100003A
:1035500053544D3332463F3F3F3F3F3F0053544D5E
:10356000333246375B347C355D780053544D33320B
:1035700046375B367C375D780000000000000000B5
:10358000CD0F0008B90F0008F50F0008E10F000883
:10359000ED0F0008D90F0008C50F0008B10F000893
:1035A00051100008000000000100000000000000B1
:1035B0006D61696E00000000D035000870240120A4
:1035C00068260120010000005919000800000000D1
:1035D00069646C650000000002000000000000004B
:1035E000F91100086112000840004000002B012082
:1035F000102B01200200000000000000030000006A
:1036000000000000A51200080000000010000000EB
:10361000202B01200000000001000000000000003D
:10362000B42D0120010102004172647550696C6F74
:10363000740025424F415244252D424C00255345EC
:103640005249414C25000000391D0008A51C000806
:1036500065110008211D00084300000060360008C5
:1036600009024300020100C0320904000001020205
:1036700001000524001001052401000104240202B8
:103680000524060001070582030800FF0904010064
:10369000020A000000070501024000000705810240
:1036A0004000000012000000AC36000812011001BA
:1036B000020000400912415700020102030100000C
:1036C0000403090425424F41524425004B616B75A8
:1036D0007465463700303132333435363738394146
:1036E0004243444546000000008000000080000086
:1036F00000800000008000000000020000000400C4
:10370000000004000000040000000000091400088C
:10371000E116000889170008400040002C2E012007
:103720002C2E0120010000003C2E01208000000012
:1037300040010000050000005001802A0000000048
:10374000AAAAAAAA00010000F3FF000000000000DE
:1037500000A00A000500000100000000AAAAAAAA11
:1037600000000001FCFF000000000000000000005D
:103770000000040000000000AAAAAAAA000000009D
:10378000FFFD0000000000000000000000000040FD
:1037900000000000AAAAAAAA00000080FF7F000083
:1037A00000000000000000000001440000000000D4
:1037B000AAAAAAAA00010000FFF50000000000006C
:1037C000000000000000000000000000AAAAAAAA51
:1037D00000000000FFFF00000000000000000000EB
:1037E0000000000000000000AAAAAAAA0000000031
:1037F000FFFF0000000000000000000000000000CB
:10380000000000000A0000000000000003000000AB
:1038100000000000000000000000000000000000A8
:103820000000000000000000000000000000000098
:103830000000000000000000000000000000000088
:103840000000000000000000000000000000000078
:103850000000000000000000000000000000000068
:103860000000000000000000000000000000000058
:10387000FF00000000000000503500083F0000007D
:10388000490400005D3500083F00000051040000BD
:103890006B3500083F0000000096000000000800A3
:1038A00004000000C0360008000000000000000016
:1038B0000000000000000000000000000000000008
:00000001FF
